:02000000442892
:100008008C00030E8D000B1D3E283E21A50A031906
:10001800A60A9B1C252822082602031C2528031D46
:10002800192821082502031C252883120614861086
:10003800061186110612861206138613A501A6015B
:100048009B109B183D2824082602031C3D28031DED
:10005800312823082502031C3D2883120610861424
:10006800061586150616861606178617A501A60113
:100078009B140B110D0E83008C0E0C0E64000900EE
:10008800A0308B00C03083168100FF3085008601C8
:10009800831206148610061186110612861206139C
:1000A80086138101E830A1000330A200C430A30008
:1000B8000930A4009B146400960197011708031DDA
:1000C80095280530160203189528980199012730BC
:1000D8001902031C7528031D7B2810301802031809
:1000E8007B280000980A0319990A64006B28831278
:1000F80006169801990127301902031C8928031D47
:100108008F281030180203188F280000980A031946
:10011800990A64007F2883120612960A0319970A1F
:100128006228640095288316051685159A1183128E
:10013800051A9A151A1185191A15A00164000800E4
:100148001D08323A0319B4281D08333A0319B42894
:100158001D08343A0319B4281D08353A031DB6287A
:1001680003140800031008009F0A1A139A13831631
:1001780085151D08323A0319CB28013A0319E828D6
:10018800073A03190429013A031921293C291A17A6
:1001980002301F02031C3C291E08A100A2012108ED
:1001A800930022089400103092000310A10DA20DB4
:1001B800930D940D031CE4286430A1070318A20AC8
:1001C800920BD9289D013C299A17210893002208EF
:1001D8009400950110309200930D940D950D03181D
:1001E800F92864301502031CFC28643095020314B6
:1001F8008E0D8F0D920BF0280E089E009D013C2954
:100208001A1702301F02031C3C291E08A300A40170
:100218002308930024089400103092000310A30DC3
:10022800A40D930D940D031C1D296430A307031816
:10023800A40A920B12299D013C299A1723089300BE
:1002480024089400950110309200930D940D950D9B
:100258000318322964301502031C352964309502CD
:100268000314900D910D920B292910089E009D01F1
:10027800640008009A109A199A141A101A191A1474
:100288009A118312051A9A151A1185191A151A1E28
:100298005A299A1952299A18542956299A185629C6
:1002A800A0015A29A00A200A03191A129A1C6D29BA
:1002B8009A1D6D291A1C69291A1969299C019E0120
:1002C8009F011A169A161A179A131A186D291A19CD
:1002D8001A121A1E9A299A189A299A1D9A299C0A5A
:1002E8001A1F8F291C08093A03198F291C0303199F
:1002F8009E018312851D8F291C08083C8E00013041
:100308008F000E0803198D29900003108F0D900B94
:1003180089290F089E079A1F9A291C08093A031D64
:100328009A291B14831285191B109A131A1EDB298C
:100338009A1CDB299A19DB291C08093A031DA629EE
:100348009C01B8209A1FC7291C08083A031DAF2929
:10035800831685150800831685111C08073C8E0036
:1003680001308F000E080319BE29900003108F0D6D
:10037800900BBA290F081E058E000E088312031D64
:100388008515031985111A1FDB291C08083A031D56
:10039800DB2983168511831285119A1EDB291E0815
:1003A8009D009A12A420031C85150318851164006A
:0203B80008003B
:02400E00F63F7B
:00000001FF
